:10000000023BDAD291D2A5D2802222020EC1E709A8
:10001000F608DFFA8046E709F208DFFA803E8882B8
:100020008C83E709F0A3DFFA8032E309F608DFFAF0
:100030008078E309F208DFFA807088828C83E30914
:10004000F0A3DFFA806489828A83E0A3F608DFFAEE
:10005000805889828A83E0A3F208DFFA804C80D23C
:1000600080FA80C680D4806980F28033801080A6B8
:1000700080EA809A80A880DA80E280CA8033898210
:100080008A83ECFAE493A3C8C582C8CCC583CCF0BC
:10009000A3C8C582C8CCC583CCDFE9DEE7800D8963
:1000A000828A83E493A3F608DFF9ECFAA9F0EDFB6A
:1000B0002289828A83ECFAE0A3C8C582C8CCC583B2
:1000C000CCF0A3C8C582C8CCC583CCDFEADEE8800B
:1000D000DB89828A83E493A3F208DFF980CC88F07D
:1000E000EF60010E4E60C388F0ED2402B4040050AE
:1000F000B9F582EB2402B4040050AF2323458223D8
:1001000090005E73BB010689828A83E0225002E779
:1001100022BBFE02E32289828A83E49322BB010C84
:10012000E58229F582E5833AF583E0225006E92548
:1001300082F8E622BBFE06E92582F8E222E5822962
:10014000F582E5833AF583E49322BB010689828A2E
:1001500083F0225002F722BBFE01F322F8BB010D0F
:10016000E58229F582E5833AF583E8F0225006E935
:100170002582C8F622BBFE05E92582C8F222EF8D52
:10018000F0A4A8F0CF8CF0A428CE8DF0A42EFE22EF
:10019000C5F0F8A3E028F0C5F0F8E58215827002FA
:1001A0001583E038F022A3F8E0C5F025F0F0E582F1
:1001B000158270021583E0C838F0E822BB010A8975
:1001C000828A83E0F5F0A3E022500687F009E71960
:1001D00022BBFE07E3F5F009E3192289828A83E452
:1001E00093F5F074019322BB0110E58229F582E5B5
:1001F000833AF583E0F5F0A3E0225009E92582F87F
:1002000086F008E622BBFE0AE92582F8E2F5F0084E
:10021000E222E5832AF583E993F5F0A3E99322BB73
:10022000010789828A83020190500B09C5F027F7E4
:10023000C5F01937F722BBFE0D09F8E325F0F3C529
:10024000F019E338F322F889828A8374019325F048
:10025000C5F0F8E4933822BB010DC58229C582C5DB
:10026000833AC5830201905011C58229F808E5F050
:1002700026F618F5F0E58236F622BBFE11C5822976
:10028000F808E225F0F5F0F218E23582F222F8E5FE
:100290008229F582E5832AF58374019325F0F5F030
:1002A000E4933822F8BB0111E58229F582E5833A0F
:1002B000F583E8F0E5F0A3F0225009E92582C8F6BD
:1002C00008A6F022BBFE09E92582C8F2E5F008F293
:1002D00022E88FF0A4CC8BF0A42CFCE98EF0A42CA7
:1002E000FC8AF0EDA42CFCEA8EF0A4CDA8F08BF0F3
:1002F000A42DCC3825F0FDE98FF0A42CCD35F0FCF1
:10030000EB8EF0A4FEA9F0EB8FF0A4CFC5F02ECDBC
:1003100039FEE43CFCEAA42DCE35F0FDE43CFC22A1
:1003200075F008758200EF2FFFEE33FECD33CDCC94
:1003300033CCC58233C5829BED9AEC99E582984017
:100340000CF582EE9BFEED9AFDEC99FC0FD5F0D6F4
:10035000E4CEFBE4CDFAE4CCF9A88222B800C1B91E
:100360000059BA002DEC8BF084CFCECDFCE5F0CB5C
:10037000F97818EF2FFFEE33FEED33FDEC33FCEB95
:1003800033FB10D703994004EB99FB0FD8E5E4F950
:10039000FA227818EF2FFFEE33FEED33FDEC33FC3D
:1003A000C933C910D7059BE99A4007EC9BFCE99A31
:1003B000F90FD8E0E4C9FAE4CCFB2275F010EF2F76
:1003C000FFEE33FEED33FDCC33CCC833C810D70776
:1003D0009BEC9AE899400AED9BFDEC9AFCE899F8B1
:1003E0000FD5F0DAE4CDFBE4CCFAE4C8F922EB9FB8
:1003F000F5F0EA9E42F0E99D42F0EC6480C864802A
:100400009845F022EB9FF5F0EA9E42F0E99D42F01C
:10041000E89C45F022E86010ECA2E713FCED13FD28
:10042000EE13FEEF13FFD8F022E8600FEFC333FFA7
:10043000EE33FEED33FDEC33FCD8F122BB0107892E
:10044000828A830205DB5005E9F80205CFBBFE0571
:10045000E9F80205E789828A830205F3BB010DE50D
:100460008229F582E5833AF5830205DB5007E92509
:1004700082F80205CFBBFE07E92582F80205E7E511
:100480008229F582E5833AF5830205F3BB010789EA
:10049000828A8302051F5005E9F8020603BBFE05A8
:1004A000E9F802060F22BB010DE58229F582E583FA
:1004B0003AF58302051F5007E92582F8020603BBBF
:1004C000FE07E92582F802060F227401FF3395E04A
:1004D000FEFDFC080808E62FFFF618E63EFEF618BB
:1004E000E63DFDF618E63CFCF6227401FF3395E08C
:1004F000FEFDFCA3A3A3E02FFFF0E58215827002AE
:100500001583E03EFEF0E582158270021583E03D22
:10051000FDF0E582158270021583E03CFCF022ECD0
:10052000F0A3EDF0A3EEF0A3EFF022A8828583F014
:10053000D083D082120542120542120542120542B2
:10054000E473E493A3C583C5F0C583C8C582C8F02E
:10055000A3C583C5F0C583C8C582C822BB0107896E
:10056000828A8302052B5005E9F802061BBBFE05B3
:10057000E9F802063422D083D082F8E49370127432
:100580000193700DA3A393F8740193F5828883E41B
:1005900073740293B5F0067403936860E9A3A3A390
:1005A000A380D8EF4E6012EF60010EEDBB010B8906
:1005B000828A83F0A3DFFCDEFA2289F05007F70974
:1005C000DFFCA9F022BBFEFCF309DFFCA9F022E668
:1005D000FC08E6FD08E6FE08E6FF22E0FCA3E0FDDD
:1005E000A3E0FEA3E0FF22E2FC08E2FD08E2FE0831
:1005F000E2FF22E493FC740193FD740293FE740302
:1006000093FF22ECF608EDF608EEF608EFF622EC82
:10061000F208EDF208EEF208EFF222D083D082E485
:1006200093F608740193F608740293F60874039322
:10063000F6740473D083D082E493F208740193F2C9
:1006400008740293F208740393F27404739002B76F
:10065000E090013CF07F011259EC90013CE09002E7
:10066000B7F01240CD900135EEF0A3EFF0900135D8
:10067000E0FEA3E0FF64624E602090013CE0900247
:10068000B7F0BEFF08BFFF057EFF7FFF221240CDFF
:10069000900135EEF0A3EFF080D39002B77401F033
:1006A000E4F529900136E02529F5291240CD900185
:1006B00035EEF0A3EFF064424E70B2E02529F52943
:1006C0001240CD900135EEF0A3EFF064134E709D13
:1006D000E02529F5291240CD900135EEF0A3EFF089
:1006E000C39461EE648094804083900135E0FEA362
:1006F000E0FFD3947EEE64809480400302066DE0B8
:100700002529F529A3EEF0A3EFF0E0FF1234459080
:100710000135EEF0A3EFF0BEFF10BFFF0D90013CDE
:10072000E09002B7F07EFF7FFF22900135E070027B
:10073000A3E0600AE4900135F0A3F002065A9001AC
:1007400037E0FEA3E0FFEE6003020C2CEF249FB421
:100750001D004003020C2C90075EF8282873020746
:10076000B50207C00207CB02082002083C02085F5E
:100770000208A70208EF02092D02094902096502D1
:10078000099A0209C80209CE0209EC0209FF020A0D
:1007900020020A30020A56020A69020954020AC7F4
:1007A000020AD5020ADB020AEC020B23020B8C02BE
:1007B0000BB2020BED900138E0FF12568B020C33A6
:1007C000900138E0FF12568B020C339001977401B0
:1007D000F0A37400F0A374A3F0F9A37401F0A37460
:1007E00000F0A3E9F07B017A0079ECE4FD121BB87C
:1007F0009000EDE0FD7C00A3E0FB7A00A3E0FF9019
:100800000158E4F0A3EFF07FF3124A6B7B017A000A
:1008100079A3121A31900138E0FF12568B020C3383
:100820007B017A0079A312224E900138E0FF7B0110
:100830007A0079A37D07124F14020C339000A3E0D5
:10084000FFC39401500E125162900138E0FF12561E
:100850008B020C33900138E0FF1256AD020C33903E
:1008600000A4E0FEA3E07806C333CE33CED8F9FD72
:10087000AC067B017A0079EC9001497440F090005D
:10088000A3E0FF123F74EF7013900138E0FF7B018B
:100890007A0079EC7D40124F14020C33900138E05D
:1008A000FF1256AD020C339000A4E0FEA3E07806E0
:1008B000C333CE33CED8F9FDAC06900141ECF0A3A2
:1008C000EDF07B017A0079A69001497440F0900028
:1008D000A3E0FF123E7FEF700B900138E0FF12564D
:1008E0008B020C33900138E0FF1256AD020C3390AE
:1008F00000A3E0FFC394015010124ECBAD0790014E
:1009000038E0FF125712020C339000A3E0B4FF123C
:100910007FFF124ECBAD07900138E0FF1257120255
:100920000C33900138E0FF1256AD020C3312390F30
:1009300090013D12051F900138E0FF7B017A01799B
:100940003D7D04124F14020C339000A3E0FF123FD0
:10095000E9020C339000A3E0FF7B017A0079A71233
:10096000405B020C339000A3E090013BF0601DE07F
:10097000B4FF05124C61801790013BE0FF14F0EFCB
:10098000600D124564EF640160EE80031257CA9057
:100990000138E0FF12568B020C33900138E0FF1251
:1009A000568B7F1E7E00125969900138E0FF125667
:1009B0008B7F1E7E00125969900138E0FF12568B22
:1009C0007F011259EC125B0412339F020C33E4FFD7
:1009D000124911EF600B900138E0FF1256AD020C86
:1009E00033900138E0FF12568B020C33900138E04F
:1009F000FF7B017A0279017D0C124F14020C3378CF
:100A0000017C027D017B017A0079A37E007F0C12BC
:100A100000DE125770900138E0FF12568B020C3343
:100A2000900138E0FF9000A2E0FD125712020C3353
:100A30009000A3E01424FD5003020C33E49001392C
:100A4000F0A3F0900138E0FF7B017A0179397D0253
:100A5000124F14020C33900138E0FF12568B9000B5
:100A6000A3E0FF1241AE020C33900138E0FF1256B2
:100A70008B9000A3E0FF1241AE122E49EF3395E0B8
:100A8000FE900139F0A3EFF0642B4E600E122E4958
:100A9000EF3395E0900139F0A3EFF0900139E07069
:100AA00004A3E0642B7018900138E0FF12568B907D
:100AB0000138E0FF12568B900138E0FF12568BE4AC
:100AC000FF1241AE020C33900138E0FF12568B1238
:100AD0005AFA020C33123004020C339000A3E0FFE8
:100AE0007B017A0079A4123245020C339000A3E016
:100AF000B4FF0DD200900138E0FF12568B020C3388
:100B00009000A3E0FFC39420500E120C4A900138CD
:100B1000E0FF12568B020C33900138E0FF1256AD05
:100B2000020C339000A3E06041046003020C339098
:100B300000A4E0F47029A3E0F47024A3E0F4701F93
:100B4000A3E0B4FF1AA3E0B4FF15A3E0B4FF10A321
:100B5000E0B4FF0B900138E0FF12568B020C33908B
:100B60000138E0FF1256AD020C337B017A0079A404
:100B7000125A59EF700B900138E0FF12568B020C9D
:100B800033900138E0FF1256AD020C3312468990C3
:100B900000ECEEF0A3EFF01246289000EEEFF0909C
:100BA0000138E0FF7B017A0079EC7D03124F1402DB
:100BB0000C339000A3E0FFC394415027A3E0FCA3B3
:100BC000E0FD7B017A0079EC1254B3EF70159001CF
:100BD00038E0FF9000A3E0FD7B017A0079EC124F32
:100BE000148050900138E0FF1256AD80469000A36B
:100BF000E0FEA3E0FF900141EEF0A3EFF09000A52E
:100C0000E0FD12519EEF701A900141E0FEA3E0FF5B
:100C10009000A5E0FD12292D900138E0FF12568BBF
:100C20008011900138E0FF1256AD8007E490013743
:100C3000F0A3F0900137E0FEA3E0FF4E7003020640
:100C40005A90013CE09002B7F022900143EFF0127D
:100C500050E6900170EEF0A3EFF07B017A02790F7D
:100C6000900143E0FD7C0012575190020FE0FEA37B
:100C7000E0FFF47002EEF47003020EBEEF4E70035C
:100C8000020EBEE4900167F0900167E0FFC394217B
:100C9000503B7B017A017974900143E0FD90017C27
:100CA000EFF01254237B017A017974900170E0FC1B
:100CB000A3E0FD122D50900167E02446F582E43454
:100CC00001F583EFF0900167E004F080BB90020F24
:100CD000E0FEA3E0FF7B017A017946123588EF60E0
:100CE000187F1E7E0012596990020FE0FEA3E0FFFC
:100CF0007B017A017946123588900146E0900144E3
:100D0000F0201E74900212E020E06D900143E0FF9D
:100D10002413F582E43402F583E0FE900144E0FD03
:100D2000EE6D6054C3ED64809480404CE0FE74131B
:100D30002FF582E43402F583EEF0EE600C90017240
:100D4000746FF0A374FEF0800A900172747FF0A3B8
:100D500074FEF07B017A01796812224E900143E023
:100D6000FF90017C7401F0A37401F0A37472F07B16
:100D7000017A01796812188F900212E020E10302D3
:100D80000E1A7B017A017974900143E0FD90017C99
:100D90007402F01255397B017A017974900170E088
:100DA000FCA3E0FD122D50900144EFF0C364809449
:100DB0008040677B017A017974900143E0FD9001E6
:100DC0007C7403F01255397B017A017974900170BB
:100DD000E0FCA3E0FD122D50900145EFF0C36480CC
:100DE00094804036E0FF25E05402FF900144E05437
:100DF000014FFFF0FD90020FE0FEA3E0FF124B67F2
:100E0000EF60177F1E7E0012596990020FE0FEA36B
:100E1000E0FF900144E0FD124B67900212E020E2F7
:100E200003020EBB7B017A017974900143E0FDE47B
:100E300090017CF01255397B017A01797490017030
:100E4000E0FCA3E0FD122D50900144EFF0C364805C
:100E5000948040677B017A017974900143E0FD90B2
:100E6000017C7401F01255397B017A01797490018B
:100E700070E0FCA3E0FD122D50900145EFF0C3643B
:100E80008094804036E0FF25E05402FF900144E06A
:100E900054014FFFF0FD90020FE0FEA3E0FF124B64
:100EA00013EF60177F327E0012596990020FE0FE47
:100EB000A3E0FF900144E0FD124B137F00227F016D
:100EC00022C0E0C0F0C083C082C0D075D008C28C00
:100ED000758A3E758C5DD28C05179002B6E0600273
:100EE00014F0A2B5B392B5300616E517541C701075
:100EF000E517A2E192A492A392A292A192A0803DB2
:100F0000E517A2E39209301904A2098002A22492F3
:100F1000A0301804A2098002A22392A1301704A2D3
:100F2000098002A22192A2301604A2098002A22006
:100F300092A3301504A2098002A21F92A4301303C9
:100F40000210F4E51225E0FFE51133FEA287E43339
:100F5000FDEEF511EF4DF512309506201103125AF2
:100F6000FAA2959211AF1CAE1BAD1AAC19EC4D4E06
:100F70004F6036A290B3301A01B3401D781974FF48
:100F80001204CCEC4D4E4F7044301A09D226D227B1
:100F90007518FA8038D20A8034751C00751B0075EC
:100FA0001A00751900B21A8024A290B3301A01B346
:100FB000501B301A08E47F20FEFDFC8006E47F030E
:100FC000FEFDFC8F1C8E1B8D1A8C19B21A201A0381
:100FD0003027067E007F0180047E007F00EE4F24D4
:100FE000FFB3921FC215E517541F14602F146076CB
:100FF0001470030210E5240360030210F4E5187076
:10100000030210F41518E518600BE517A2E592A588
:1010100092A70210F4D2A7D2A50210F420143E0524
:1010200016E51670020515D39457E515940240068F
:10103000751500751600E5168515F0120576105524
:1010400000001059000F104E024F0000105F308159
:101050000EC281800AD21D8006D2818002D222A2D5
:101060002292210210F4201273E5124511600EE560
:10107000122401FFE435114F6003D38001C3920FA6
:1010800030050B200F08751303751484800C2005A0
:1010900009300F0675130175142CE51445136036DD
:1010A000E5141514700215131445137029A20730A6
:1010B0000F01B3401FA20FB39207A207E433FFE56D
:1010C0001870047E0180027E00EE5F60097518FAD8
:1010D000D20B8002D20EA20F92058002C207A20795
:1010E000B39223800FE51730E502D201051FE51FFB
:1010F0007002D204D0D0D082D083D0F0D0E03212AF
:1011000052801226FD9002B77401F012480390003D
:10111000A2EFF0603C24FD601114601514601924E6
:101120000370237F0212562380277F0312562380E9
:10113000207F041256238019E4FB7D017F05123ABB
:10114000C0125805800B9000A27406F07F0A125658
:1011500023E4900158F0A3F0FBFA7D01FC7FF1122B
:101160004A6B9002B77402F01259AD1259FF301059
:10117000031243627D017FFF1239A1E4FF1241AEE9
:10118000300C24301021124362C2A57FF47E01127C
:101190005969D2A5E4900158F0A3F0FBFA7D02FC56
:1011A0007FF1124A6BD200200C14201011E4900140
:1011B00058F0A3F0FBFA7D03FC7FF1124A6B124852
:1011C00060300414C20420020F124803EF600924A7
:1011D000FB60058000125B0412390F90012D12058F
:1011E0001F900265E0FCA3E0FDA3E0FEA3E024164F
:1011F000FFEE34FCFEED34FFFDEC34FFFC90012DDE
:10120000E0F8A3E0F9A3E0FAA3E0FBD31204044062
:101210000BE4FB7D017F05123AC08047E47F03FEAB
:10122000FDFC900265E0F8A3E0F9A3E0FAA3E0FB7F
:101230001202D1E47B04FAF9F812035C90012DE06C
:10124000F8A3E0F9A3E0FAA3E0FBD3120404400BF7
:101250007B01E4FD7F05123AC08008E4FBFD7F05B9
:10126000123AC0A210B3920C300C18E4FB7D017F3F
:1012700002123AC09000A27401F01255FD124DA066
:1012800002117BE4FBFD7F02123AC0E49000A2F061
:10129000124DA08014E51EC394205009AF1E120CFD
:1012A0004A051E80F0151EC20074082510F510C3F3
:1012B00094204003E4F510E5102407FDAF10122B35
:1012C00040EF6003125B0430012BC201E490013156
:1012D000F0051EE51EC394204003E4F51EE51EC381
:1012E00094205005AF1E120C4A900131E004F0E04A
:1012F000C3940340DC7F967E001259691248B912EC
:10130000130602117B227B017A017943124DEC7B9B
:10131000017A01793412224E12390F90013F1205E1
:101320001F7B017A0279331247477F2A12521290AB
:101330000132741BF0FF1256F1900132E02529F5BD
:1013400029E4A3F07B0190013C04F0A37401F0A315
:10135000743FF090013CE0FBA3E0FAA3E0F9120136
:1013600004FF1256F190013CE0FBA3E475F001127A
:1013700001A6A9F0FA1201042529F529900133E00C
:1013800004F0E0C3940440CBE4900133F07B01907F
:10139000013C04F0A37401F0A37434F090013CE02C
:1013A000FBA3E0FAA3E0F9120104FF1256F1900149
:1013B0003CE0FBA3E475F0011201A6A9F0FA1201CA
:1013C000042529F529900133E004F0E0C394074097
:1013D000CBE4900133F07B0190013C04F0A3740254
:1013E000F0A37433F090013CE0FBA3E0FAA3E0F932
:1013F000120104FF1256F190013CE0FBA3E475F0EA
:10140000011201A6A9F0FA1201042529F52990017B
:1014100033E004F0E0C3940440CBE4900133F07B6C
:101420000190013C04F0A37402F0A37465F09001F4
:101430003CE0FBA3E0FAA3E0F9120104FF1256F12D
:1014400090013CE0FBA3E475F0011201A6A9F0FABB
:101450001201042529F529900133E004F0E0C3943A
:101460000440CBE4900133F07B0190013C04F0A3F5
:101470007401F0A37447F090013CE0FBA3E0FAA3F1
:10148000E0F9120104FF1256F190013CE0FBA3E4E5
:1014900075F0011201A6A9F0FA1201042529F52917
:1014A000900133E004F0E0C3940440CBE4900133B6
:1014B000F07B0190013C04F0A37401F0A37443F0AD
:1014C00090013CE0FBA3E0FAA3E0F9120104FF1253
:1014D00056F190013CE0FBA3E475F0011201A6A9CE
:1014E000F0FA1201042529F529900133E004F0E017
:1014F000C3940440CBAF291256F11258DA7F01127F
:1015000059EC22900148EEF0A3EFF0A3EDF0C39464
:101510002040037F012290014AE075F002A424627A
:10152000F9740035F0FA90014C7401F0A3EAF0A3CD
:10153000E9F0302A1E90014CE0FBA3E0FAA3E0F9A9
:10154000120104900041F090000112011D90004032
:10155000F0801C90014CE0FBA3E0FAA3E0F99000BE
:101560000112011D900041F0120104900040F09022
:101570000041E0C394FA500A900040E0FDC394FAA1
:1015800040037F0222900148E0FEA3E0FF12558A4B
:10159000900040E0FD7C00900148E0FB7A00E49080
:1015A0000158F0900149E0900159F07FF5124A6B23
:1015B000E490014BF090014BE0FFC3942040030204
:1015C00016E690014AE0FEEF6E70030216DDEF753D
:1015D000F002A42462F9740035F0FA7B0190014C0A
:1015E000EBF0A3EAF0A3E9F0120104FFC394FA4080
:1015F000030216DD90014CE0FBA3E0FAA3E0F990B2
:10160000000112011DFEC394FA40030216DD900092
:1016100041E0B5071A900040E0B50613900148E09C
:10162000FEA3E0FF90014BE0FD1253200216DD9077
:10163000014CE0FBA3E0FAA3E0F990000112011DC8
:10164000FF900041E0B5071D120104FF900040E04B
:10165000B50712900148E0FEA3E0FF90014BE0FDCA
:101660001252EB807890014CE0FBA3E0FAA3E0F982
:10167000120104FF900040E0B50712900148E0FE1F
:10168000A3E0FF90014BE0FD1252EB805090014C23
:10169000E0FBA3E0FAA3E0F990000112011DFF9026
:1016A0000040E0B50712900148E0FEA3E0FF900182
:1016B0004BE0FD1253208025200312900148E0FEEC
:1016C000A3E0FF90014BE0FD1253558010900148BC
:1016D000E0FEA3E0FF90014BE0FD1252B690014BFB
:1016E000E004F00215B57F002290019A12051F90C8
:1016F000019EEBF0A3EAF0A3E9F090019AE0FCA3CD
:10170000E0FDA3E0FEA3E0FFE4EFF4049001A2F00B
:10171000600AE0FF9001A1E0D39F506790019AE03A
:10172000FCA3E0FDA3E0FEA3E0FF12413E90019A7E
:10173000E0FCA3E0FDA3E0FEA3E0FF9001A1E0FB3D
:101740009001A7E4F0A3EBF090019EE0F9A3E0FA8A
:10175000A3E09001A9C9F0A3EAF0A3E9F01249BF00
:1017600090019AE0FCA3E0FDA3E0FEA3E0FF124F8E
:101770005B90019AE0FCA3E0FDA3E0FEA3E0FF1272
:1017800055632290019AE0FCA3E0FDA3E0FEA3E0F4
:10179000FF12413E90019AE0FCA3E0FDA3E0FEA30E
:1017A000E0FF9001A2E0FB9001A7E4F0A3EBF09032
:1017B000019EE0F9A3E0FAA3E09001A9C9F0A3EA31
:1017C000F0A3E9F01249BF90019AE0FCA3E0FDA369
:1017D000E0FEA3E0FF124F5B90019AE0FCA3E0FD66
:1017E000A3E0FEA3E0FF12556390019AE0F8A3E0A6
:1017F000F9A3E0FAA3E0FB9001A2E0FFE4FCFDFE08
:10180000EB2FFFEE3AFEED39FDEC38FC90019A1219
:10181000051F90019AE0FCA3E0FDA3E0FEA3E0FF1A
:1018200012413E9001A2E0FF9001A1E0C39F900110
:10183000A8F0E494009001A7F090019EE0FBA3E0E3
:10184000FAA3E0F99001A2E07E00E92FF9EE3AFA5E
:101850009001A9EBF0A3EAF0A3E9F090019AE0FC73
:10186000A3E0FDA3E0FEA3E0FF1249BF90019AE0D0
:10187000FCA3E0FDA3E0FEA3E0FF124F5B90019A02
:10188000E0FCA3E0FDA3E0FEA3E0FF12556322907D
:101890000178EFF0A3EBF0A3EAF0A3E9F07B017A83
:1018A000017987124DECEF60037F0222900178E00E
:1018B000FDA3E0F9A3E0FAA3E0900197C9F0A3EA41
:1018C000F0A3E9F090017CE0F9A3E0FAA3E0900135
:1018D0009AC9F0A3EAF0A3E9F07B017A01797F12BB
:1018E0001BB8900187E0FCA3E0FDA3E0FEA3E0FFAE
:1018F0007B017A01797F124E379001871204EA90BA
:101900000265E0F8A3E0F9A3E0FAA3E0FBD3120438
:1019100004500A90018712052B0000000090018BF3
:10192000E0FCA3E0FDA3E0FEA3E0FF900187E0F868
:10193000A3E0F9A3E0FAA3E0FBC3120404600302EE
:101940001A2590018BE0FCA3E0FDA3E0FEA3E0FFDD
:101950007B017A01797F125067900183E064F06027
:101960001690017F74FFF090018374F0F0E4A3F00F
:10197000A3F0A304F08016900186E004F0700E90AE
:101980000185E004F07006900184E004F090018B82
:10199000E0FCA3E0FDA3E0FEA3E024E8FFEE3403B7
:1019A000FEE43DFDE43CFC90018B12051F900265B6
:1019B000E0FCA3E0FDA3E0FEA3E0FF90018BE0F8D4
:1019C000A3E0F9A3E0FAA3E0FBC3120404402E90C5
:1019D000018BE0FCA3E0FDA3E0FEA3E0FF90026525
:1019E000E0F8A3E0F9A3E0FAA3E0FBEF9BFFEE9A97
:1019F000FEED99FDEC98FC90018B12051F90018B78
:101A0000E0FCA3E0FDA3E0FEA3E0FF7B017A017907
:101A10007F124E3790018FE07002A3E070079001B3
:101A20008FF0A304F07B017A0179871251DA7F00ED
:101A300022900143EBF0A3EAF0A3E9F0900143E028
:101A4000FBA3E0FAA3E0F9120104D394634004E499
:101A500012014A900143E0FBA3E0FAA3E0F99000F1
:101A60000112011DFFD3940C5006EFC394015008DE
:101A7000900001740112015C90000212011DFFD35D
:101A8000941F5006EFC39401500890000274011295
:101A9000015C90000312011DD394174007900003CE
:101AA000E412015C90000412011DD3943B400790A6
:101AB0000004E412015C90000512011DD3943B4028
:101AC00007900005E412015C90000612011DD394FA
:101AD000064007900006E412015CE490028FF0A338
:101AE000F0900143E0FBA3E0FAA3E0F990000512B7
:101AF000011DFF1259D8900291EFF0900143E0FBD5
:101B0000A3E0FAA3E0F990000412011DFF1259D8D6
:101B1000900292EFF0900143E0FBA3E0FAA3E0F91A
:101B200090000312011DFF1259D8900293EFF0901C
:101B30000143E0FBA3E0FAA3E0F990000212011DCB
:101B4000FF1259D8900143E0FBA3E0FAA3E0F91299
:101B50000104FEC4333354C04F900294F09000014E
:101B600012011DFF1259D8900143E0FBA3E0FAA334
:101B7000E0F990000612011DFEC43354E04F9002BC
:101B800095F090019C7401F0A37402F0A3748FF09F
:101B9000E4FB7D077FA012538A900143E0F9A3E0A4
:101BA000FAA3E090019CC9F0A3EAF0A3E9F07B3A24
:101BB0007D017FA012538A22900193EBF0A3EAF0FB
:101BC000A3E9F0900193E0FBA3E475F0011201A6F4
:101BD000A9F0FAED12014A900197E0FBA3E0FAA305
:101BE000E0F990000212011DFFC313540FFF900093
:101BF0000112011DFEC454F04FFF900193E0FBA3BE
:101C0000E475F0011201A6A9F0FAEF12014A900161
:101C100097E0FBA3E0FAA3E0F990000212011DFF98
:101C2000C43333335480FF120104FEC433335440B1
:101C30004FFF90000412011D543F4FFF900193E0AD
:101C4000FBA3E475F0011201A6A9F0FAEF12014A14
:101C5000900197E0FBA3E0FAA3E0F99000051201E0
:101C60001D75F00A84FFC43354E0FF900003120195
:101C70001D541F4FFF900193E0FBA3E475F0011288
:101C800001A6A9F0FAEF12014A90019AE0FBA3E441
:101C900075F0011201A6A9F0FA120104FF90019358
:101CA000E0FBA3E475F0011201A6A9F0FAEF12011E
:101CB0004A90019AE0FBA3E475F0011201A6A9F095
:101CC000FA120104FF900193E0FBA3E475F0011206
:101CD00001A6A9F0FAEF12014A90019AE0FBA3E4F1
:101CE00075F0011201A6A9F0FA120104FF90019308
:101CF000E0FBA3E475F0011201A6A9F0FAEF1201CE
:101D00004A90019AE0FBA3E0FAA3E0F9120104FF74
:101D1000900193E0FBA3E0FAA3E0F9EF12014A225D
:101D2000900159EEF0A3EFF0A3EDF0A3EBF0A3EADE
:101D3000F0A3E9F07F011259ECE49002B7F01240F1
:101D4000CD900169EEF0A3EFF0900169E0FCA3E013
:101D5000FDBCFF06BDFF037F0122ED64234C70DE56
:101D60009001D1F090016AE0FF9001D1E02FF012D4
:101D700040CD900169EEF0FCA3EFF0FD900159E039
:101D8000B505C6E4B504C290016AE0FF9001D1E058
:101D90002FF01240CD900169EEF0A3EFF090015AC0
:101DA000E0B507A5E4B506A190016AE0FF9001D176
:101DB000E02FF01240CD90015FE0FBA3E0FAA3E03A
:101DC000F9EF12014A90015FE0FBA3E0FAA3E0F90A
:101DD000120104FF9001D1E02FF01240CD9001627A
:101DE000E0FBA3E0FAA3E0F9EF12014A900162E000
:101DF000FBA3E0FAA3E0F9120104FE9001D1E02E6A
:101E0000F090015BE0FFEED39F40037F0222900140
:101E100065EEF090015CE0F9A3E0FAA3E0900166C2
:101E2000C9F0A3EAF0A3E9F0900165E0D394004083
:101E30003C1240CD900169EEF0A3EFF0F47002EE99
:101E4000F47003021D4990016AE0FF9001D1E02F78
:101E5000F0900166E0FBA3E475F0011201A6A9F081
:101E6000FAEF12014A900165E014F080BB1240CDF8
:101E7000900169EEF0A3EFF09001D1E06F7001EEF8
:101E80006003021D497F0022125A489001ADE0FC18
:101E9000A3E0FDA3E0FEA3E0FF780F120415EFE43A
:101EA000125A489002B3E024F8600B24E8606124E1
:101EB0001E6003021FCA9001ADE0FCA3E0FDA3E099
:101EC000FEA3E0FF7818120415EC4D4E4F602390EE
:101ED00001ADE0FCA3E0FDA3E0FEA3E0FF78071264
:101EE0000415EF54FEFFE4EF4401FFE4125A4802E8
:101EF0001FCF9001ADE0FCA3E0FDA3E0FEA3E0FF57
:101F00007807120415EF54FEFFE4125A48021FCF5F
:101F10009001ADE0FCA3E0FDA3E0FEA3E0FF781894
:101F2000120415EC4D4E4F60539001ADE0FCA3E060
:101F3000FDA3E0FEA3E0FF7807120415EF54FCFFB9
:101F4000E4FEFDFCEF4402FFE4C004C005C006C08F
:101F5000079001ADE0FCA3E0FDA3E0FEA3E0FF7865
:101F600008120415EF5401FFE4D003D002D001D0D1
:101F700000EB4FFFEAE9E8125A4880539001ADE0C8
:101F8000FCA3E0FDA3E0FEA3E0FF7808120415EF38
:101F90005401FFE4FEFDFCC004C005C006C007906C
:101FA00001ADE0FCA3E0FDA3E0FEA3E0FF78071293
:101FB0000415EF54FCFFE4D003D002D001D000EFB1
:101FC0004BFFEAE9E8125A4880057F011258059054
:101FD00001ADE0FCA3E0FDA3E0FEA3E0FFE4125AA4
:101FE0004822900197EBF0A3EAF0A3E9F0A31205D1
:101FF0001F90019AE0FCA3E0FDA3E0FEA3E0FFE454
:10200000EFF404FF90019FF090019EE0D39F5040B9
:1020100090019AE0A3E0A3E0A3E0FF12413E90010B
:102020009AE0FCA3E0FDA3E0FEA3E0FFA3E0FB90A9
:1020300001A4E4F0A3EBF0900197E0F9A3E0FAA388
:10204000E09001A6C9F0A3EAF0A3E9F0124BBB228D
:1020500090019AE0FCA3E0FDA3E0FEA3E0FF1241A3
:102060003E90019AE0FCA3E0FDA3E0FEA3E0FF9018
:10207000019FE0FB9001A4E4F0A3EBF0900197E056
:10208000F9A3E0FAA3E09001A6C9F0A3EAF0A3E95E
:10209000F0124BBB90019AE0F8A3E0F9A3E0FAA399
:1020A000E0FB90019FE0FFE4FCFDFEEB2FFFEE3A2A
:1020B000FEED39FDEC38FC90019A12051F90019A53
:1020C000E0FCA3E0FDA3E0FEA3E0FF12413E90018F
:1020D0009FE0FF90019EE0C39F9001A5F0E4940073
:1020E0009001A4F0900197E0FBA3E0FAA3E0F9903F
:1020F000019FE07E00E92FF9EE3AFA9001A6EBF09D
:10210000A3EAF0A3E9F090019AE0FCA3E0FDA3E0CC
:10211000FEA3E0FF124BBB22900271EFF0E4FF122E
:1021200059EC7BFF7A3B795E1250267FD07E0712F6
:1021300059697BFF7A3B79621250267FD07E071265
:1021400059697BFF7A3B79661250267FD07E071251
:1021500059697BFF7A3B796A1250267FD07E07123D
:1021600059697BFF7A3B7979125026E490027DF021
:1021700090024BE0FF90027DE0FD3395E0FCC3ED63
:102180009F7480F86C98400302224BE4FF1259ECD4
:102190007BFF7A3B79551250267BFF7A3B796E1292
:1021A00050267F011259EC7B017A02793790024A5E
:1021B000E09002A5F07D101246E8900271E0FF6009
:1021C00004640170397B017A0279727D011236B89C
:1021D0007B017A0279721259C390028DEEF0A3EF5F
:1021E000F090028A7401F0A37402F0A37472F07B81
:1021F000017A027937124433EF60037F01229002A3
:1022000071E0FF6004640270397B017A0279727DAB
:10221000021236B87B017A0279721259C390028D8C
:10222000EEF0A3EFF090028A7401F0A37402F0A321
:102230007472F07B017A027937124433EF60037FC6
:10224000022290027DE004F00221707F00229001C2
:1022500080EBF0A3EAF0A3E9F07B017A0279919098
:10226000019B7402F07D057FA012428C900291E0E8
:10227000900183F07B017A02799190019B7402F0C6
:102280007D057FA012428C900291E0FF900183E0D7
:102290006F60137B017A02799190019B7402F07D4B
:1022A000057FA012428C7B017A01798390019B7497
:1022B0003AF07D017FA012428C900291E0547FFFA2
:1022C000125A99900180E0FBA3E0FAA3E0F9900094
:1022D00005EF12015C900292E0547FFF125A999030
:1022E0000180E0FBA3E0FAA3E0F9900004EF120103
:1022F0005C900293E0543FFF125A99900180E0FBFA
:10230000A3E0FAA3E0F9900003EF12015C900294BD
:10231000E0543FFF125A99900180E0FBA3E0FAA33A
:10232000E0F9900002EF12015C900295E0541FFF6B
:10233000125A99900180E0FBA3E0FAA3E0F9900023
:1023400001EF12015C900294E0FFC413135403FFE9
:10235000900183E0FE5403B50706EE12014A8005A2
:10236000EE0412014A900295E0FFC4135407FF9057
:102370000180E0FBA3E0FAA3E0F9900006EF120170
:102380005C22900296EEF0A3EFF0A3EDF0FF7B014C
:102390007A02799A1258A630291290029AE0900097
:1023A00041F090029BE0900040F0801090029BE092
:1023B000900041F090029AE0900040F0900296E088
:1023C000FEA3E0FF900040E0FD12558AE4900299E0
:1023D000F0900299E0FFC394FA40030224AA90020D
:1023E00098E0FEEF6E70030224A17B017A02799AD5
:1023F0001258A690029AE0FFC394FA40030224A167
:10240000A3E0FEC394FA40030224A1900041E0B58A
:102410000719900040E0B50612900296E0FEA3E096
:10242000FF900299E0FD125320807690029BE0FF1E
:10243000900041E0B5071E90029AE0FF900040E056
:10244000B50712900296E0FEA3E0FF900299E0FD2E
:102450001252EB804C90029AE0FF900040E0B507EA
:1024600012900296E0FEA3E0FF900299E0FD125266
:10247000EB802E90029BE0FF900040E0B5071290A9
:102480000296E0FEA3E0FF900299E0FD1253208047
:1024900010900296E0FEA3E0FF900299E0FD125337
:1024A00055900299E004F00223D17F002290014B65
:1024B000EFF0A3EDF090014BE02400F582E434004E
:1024C000F583E090014EF0C3942040037F012290F9
:1024D000014CE060067C007D0180047C007D009062
:1024E000014EE0FF900158E4F0A3EFF0E4FBFA7F27
:1024F000F6124A6BE490014DF090014DE0FFC39459
:1025000020503A90014BE0FEEF6E602974002FF5E9
:1025100082E43400F583E0FE90014EE0FDEEB50567
:102520001490014CE06003D38001C3922A900153C0
:10253000EFF012512490014DE004F080BC90014C6A
:10254000E070030225D3E4A3F090014FF090014F17
:10255000E0FF90014DE0D39F504DE4FF74202FF534
:1025600082E43400F583E0FE90014EE0FDEEB50517
:1025700017A3E0C394205010E0FE04F074422EF53F
:1025800082E43400F583EFF00FEFB420CF90014DDB
:10259000E02442F582E43400F583E090014EF090AF
:1025A000014DE004F080A6E490014DF090014FE071
:1025B000FF90014DE0FEC39F501974422EF582E456
:1025C0003400F583E0FF7D01123EFD90014DE004F3
:1025D000F080D97F0022900183EEF0A3EFF0A3ED0D
:1025E000F0A3EBF07F011259ECE49002B7F0124037
:1025F000CD90018EEEF0A3EFF090018EE0FCA3E011
:10260000FDBCFF06BDFF037F0122ED64034C70DEBD
:102610009001D1F090018FE0FF9001D1E02FF012F6
:1026200040CD90018EEEF0FCA3EFF0FD900183E031
:10263000B505C6E4B504C290018FE0FF9001D1E07A
:102640002FF01240CD90018EEEF0A3EFF0900184B8
:10265000E0B507A5E4B506A190018FE0FF9001D198
:10266000E02FF01240CD90018EEEF0A3EFF090013C
:1026700085E06F7001EE708190018FE0FF9001D1D5
:10268000E02FF0900186E090018DF0900187E0F955
:10269000A3E0FAA3E0A3C9F0A3EAF0A3E9F0900154
:1026A0008DE0D39400403B1240CD90018EEEF0A31C
:1026B000EFF0BEFF06BFFF037F012290018FE0FF16
:1026C0009001D1E02FF090018AE0FBA3E475F001C6
:1026D0001201A6A9F0FAEF12014A90018DE014F060
:1026E00080BC1240CD90018EEEF0A3EFF09001D1AE
:1026F000E06F7001EE60030225F97F0022D21375AE
:1027000080FF7590FF75A0FF75B0FFE4F510D20152
:10271000751EFFF51FD204C208C226C20AC21CC21F
:102720000DC20BC20EFBFD7F01123AC0E40F123A3C
:10273000C0E40F123AC0E40F123AC0E40F123AC0DC
:10274000D2A5D2A7751502751644D222D281C21D18
:10275000D20FD205C207E4F513F5147455F511F53F
:1027600012A2959211A290B3921AC227E4751C0886
:10277000F51BF51AF519D20CC206FF7F2090021343
:1027800074FFF0A3DFFC7F201259807F011259EC07
:10279000125A7AE4FF1241AED2B77F1E7E00125960
:1027A0006920B73D20B71A7F0A7E0012596920B709
:1027B000077F0112580580F67F0A7E001259698052
:1027C000E3124FE41255D71256697FFF125162127D
:1027D00057CA1250A712578E7F3C7E00125969804B
:1027E00006124FE41255D712588CEF60227FF47E08
:1027F000011259697F031258057FF47E011259694D
:102800007F031258057FE87E031259691256691238
:102810005B279002C37408F0C21322900150EBF0C2
:10282000A3EAF0A3E9F07B017A017953124DEC9011
:102830000157E0FCA3E0FDA3E0FEA3E0FF900153FD
:10284000E0F8A3E0F9A3E0FAA3E0FBD3120404400C
:102850006E900150E0FBA3E0FAA3E0F912043C9073
:102860000153E0F8A3E0F9A3E0FAA3E0FBC31204EC
:10287000044022900150E0FBA3E0FAA3E0F9120427
:102880003C900157E0F8A3E0F9A3E0FAA3E0FBD302
:102890001204044015900153E0FCA3E0FDA3E0FE08
:1028A000A3E0FF90026D12051F22900150E0FBA3F0
:1028B000E0FAA3E0F912043C90026D12051F229089
:1028C0000150E0FBA3E0FAA3E0F912043C900153AD
:1028D000E0F8A3E0F9A3E0FAA3E0FBC3120404507C
:1028E00037900150E0FBA3E0FAA3E0F912043C901A
:1028F0000157E0F8A3E0F9A3E0FAA3E0FBD3120448
:10290000044015900153E0FCA3E0FDA3E0FEA3E02A
:10291000FF90026D12051F22900150E0FBA3E0FA28
:10292000A3E0F912043C90026D12051F22900143AE
:10293000EEF0A3EFF0A3EDF0C394FA4007E0F460EB
:10294000037F0222900145E0FD7C00900143E0FB03
:102950007A00E4900158F0900144E0900159F07F32
:10296000F5124A6BE4900146F0900146E0FFC394F3
:10297000204003022A34EF75F002A42462F97400A7
:1029800035F0FA7B01A3EBF0A3EAF0A3E9F0120122
:1029900004C394FA4003022A2B900147E0FBA3E012
:1029A000FAA3E0F990000112011DC394FA507C9043
:1029B0000145E0B4FF12900143E0FEA3E0FF900167
:1029C00046E0FD1252B68063900147E0FBA3E0FAB7
:1029D000A3E0F990000112011DFF900145E0B50749
:1029E00012900143E0FEA3E0FF900146E0FD125388
:1029F000208038900147E0FBA3E0FAA3E0F9120140
:102A000004FF900145E0B50712900143E0FEA3E00A
:102A1000FF900146E0FD1252EB8010900143E0FE72
:102A2000A3E0FF900146E0FD125355900146E004FB
:102A3000F00229697F0022302807209103022B2011
:102A400022A29150028001C34003022B3FC280E4C6
:102A5000900158F0A3F0FBFA7D01FC7FF4124A6B61
:102A60007FC87E00125969E4FF1221189002C5EF59
:102A7000F07003022B0E125ACD40199002C5E0FBF4
:102A80007A00E4900158F0A3F07D02FC7FF4124A32
:102A90006BD22822D2A57FD07E07125969C2A59099
:102AA00002C5E0FB7A00E4900158F0A3F07D03FC3E
:102AB0007FF4124A6B9002C5E0FF122F35EF703A97
:102AC0009002C5E0FF1221189002C5E0FEB507167E
:102AD000EEFB7A00E4900158F0A3F07D02FC7FF455
:102AE000124A6BD22822E4900158F0A3F07B01FA3D
:102AF0007D04FC7FF4124A6B8026E4900158F0A319
:102B0000F07B02FA7D04FC7FF4124A6B8012E490A1
:102B10000158F0A3F07B01FA7D04FC7FF4124A6BAC
:102B2000D2A57FE87E031259697BFF7A3B79751243
:102B30005026D2807F647E00125969C2A5C2282225
:102B4000900132EFF0A3EDF0C394204003741FF026
:102B50007B017A01793E12224E900132E0900134DD
:102B6000F0900133E0FFA3E0FD3395E0FCD3ED9F4F
:102B70007480F86C984003022C457B017A02790F2F
:102B800012575190020FE0FEA3E0FFF47002EEF442
:102B90007003022C3CEF4E7003022C3C90020FE0BD
:102BA000FEA3E0FF7B017A01793612319690013560
:102BB000EFF07070A3E054F0606A900134E0FF120F
:102BC0003A32900134E0FF90017C7401F0A374016B
:102BD000F0A37436F07B017A01793E12188F9002CF
:102BE0000FE0FEA3E0FF7D01124E81EF60177F0A28
:102BF0007E0012596990020FE0FEA3E0FF7D0112F2
:102C00004E81EF601F900134E0FF7B017A0179363D
:102C1000123C66900134E0FF7B017A017936123470
:102C2000E8022B9C900135E0600A900134E0FF122D
:102C300037E48008900134E0FF123A32900134E02A
:102C400004F0022B617F0022094300A00954009F79
:102C50000966009E0977009D0989009C099B009BDD
:102C600009AD009A09BF009909D2009809E40097BC
:102C700009F700960A0A00950A1D00940A3000938D
:102C80000A4300920A5700910A6B00900A7F008F56
:102C90000A93008E0AA7008D0ABB008C0AD1008B14
:102CA0000AE7008A0AFE00890B1400880B2B0087B4
:102CB0000B4300860B5C00850B7500840B8E008334
:102CC0000BA700820BC100810BDB00800BF6007F9D
:102CD0000C10007E0C2B007D0C47007C0C64007BEC
:102CE0000C81007A0C9E00790CBB00780CDB00771D
:102CF0000CFB00760D1B00750D3B00740D5B007323
:102D00000D7D00720D9F00710DC200700DE4006F0B
:102D10000E07006E0E2C006D0E51006C0E76006BCF
:102D20000E9B006A0EC100690EE900680F11006772
:102D30000F3900660F6100650F8900640FB30063EF
:102D40000FDE00621009006110340060105F005F48
:102D5000900178EBF0A3EAF0A3E9F0A3ECF0A3ED87
:102D6000F0A374FFF0900178E0FBA3E0FAA3E0F990
:102D70009000021201E7FFAEF04E7003022E43C333
:102D8000EF9410EE94274003022E431201BCFFAED5
:102D9000F0C39410EE94274003022E4390000212D9
:102DA00001E72FFFEE35F0FEC3EF9410EE942740BD
:102DB00003022E43900178E0A3E0A3E01201BCFDE2
:102DC000ACF07B017A01797E12582290017EE0FE00
:102DD000A3E0FFEE547FFCEF4C7068EEC4131313B6
:102DE000540190017DF0900178E0FBA3E0FAA3E0AC
:102DF000F990000274FFF5F012025745F06044901C
:102E00000178E0FBA3E0FAA3E0F9E475F001120217
:102E10001FADF0FC7B017A01797E12582290017E71
:102E2000E0FEA3E0FFEE547FFCC390017CE09F90A6
:102E3000017BE09C400DEEC4131313540190017DFF
:102E4000F080A390017DE0FF227F011259EC9002F7
:102E5000B77401F0E4900145F0A3F01240CD900169
:102E600043EEF0A3EFF064624E602E900143E0B4B5
:102E7000FF08A3E0B4FF037FFF22900146E004F0C7
:102E80007006900145E004F0C3900146E0940A907A
:102E90000145E06480948040C2900143E07004A347
:102EA000E0646260037F2D221240CD900143EEF07A
:102EB000A3EFF064424E60037F2D221240CD9001BB
:102EC00043EEF0A3EFF064134E60037F2D22124017
:102ED000CD900143EEF0A3EFF064744E60037F2DBC
:102EE000221240CD900143EEF0A3EFF0BEFF06BFEB
:102EF000FF037F2D22900144E0242BFFE43401E402
:102F0000900147F0EFA3F01240CD900143EEF0A303
:102F1000EFF0BEFF06BFFF037F2D22900147E0FECA
:102F2000A3E0FF900143E06E7003A3E06F60037FB6
:102F30002D227F2B22900253EFF0E4A3F090024C5D
:102F4000E0FF900254E0FD3395E0FCC3ED9F7480F8
:102F5000F86C984003023003E4FF1259EC7B017ACD
:102F6000027955900253E0FD12374E900260E0FB6B
:102F7000A3E0FAA3E0F9745512014A7BFF7A3B798A
:102F800051125249900260E0FBA3E0FAA3E0F9126B
:102F900001046018900260E0A3E475F0011201A63C
:102FA000A9F0FA120104FF1256F180D87BFF7A3B98
:102FB00079551250267F011259EC7B017A0279373C
:102FC00090024BE09002A5F07D101246E87BFF7A5C
:102FD0003B79561259C390028DEEF0A3EFF09002A8
:102FE0008A74FFF0A3743BF0A37456F07B017A025D
:102FF0007937124433EF7002FF22900254E004F05C
:10300000022F3D227B017A017944124DEC7F771229
:103010005212E4900143F075260175270275286568
:10302000AB26AA27A928120104FF1256F1AB2605E8
:1030300028E528AA277002052714F912010425297A
:10304000F529900143E004F0E0C3940440D2E490F9
:103050000143F0752601752701752844AB26AA2780
:10306000A928120104FF1256F1AB260528E528AA6B
:10307000277002052714F91201042529F52990016A
:1030800043E004F0E0C3940440D2E4900143F075BF
:103090002601752701752848AB26AA27A928120101
:1030A00004FF1256F1AB260528E528AA2770020571
:1030B0002714F91201042529F529900143E004F0B1
:1030C000E0C3940440D2AF291256F11258DA7F2B94
:1030D00022900159EEF0A3EFF0A3EDF0A3EBF0E4A2
:1030E000FF1259ECE49001D1F07F211256F19001CA
:1030F000D1E02421F0900159E0FF1256F1900159DE
:10310000E0FF9001D1E02FF090015AE0FF1256F15C
:1031100090015AE0FF9001D1E02FF090015BE0FFB9
:103120001256F190015BE0FF9001D1E02FF0900189
:103130005CE0FF1256F190015CE0FF9001D1E02FBE
:10314000F0900160EFF0900160E0D394004039907E
:10315000015DE0FBA3E0FAA3E0F9120104FF1256BF
:10316000F190015DE0FBA3E0FAA3E0F9120104FF96
:103170009001D1E02FF090015EE475F00112019012
:10318000900160E014F080BE9001D1E0FF1256F192
:103190007F061256F122900146EEF0A3EFF0A3EB6A
:1031A000F0A3EAF0A3E9F090014D7403F09001461A
:1031B000E0FEA3E0FFE4FB7D41123E00900146E00B
:1031C000FEA3E0FF9001877401F0A37401F0A374E3
:1031D0004BF07B027D411225D6EF705790014BE0FA
:1031E000FF900148E0FBA3E475F0011201A6A9F0ED
:1031F000FAEF12014A90014CE0FF900148E0FBA376
:10320000E475F0011201A6A9F0FAEF12014A90014B
:1032100048E0FBA3E475F0011201A6A9F0FAE4125C
:10322000014A900148E0FBA3E0FAA3E0F9E41201AF
:103230004AFF2290014DE014F0E0D39400400302D5
:1032400031AD7F0122900143EFF0A3EBF0A3EAF050
:10325000A3E9F07F78125212900143E0FF14F0EFDF
:1032600070030232EA9001567401F0A37401F0A3D6
:103270007448F0900144E0FBA3E0FAA3E0F9124D9A
:1032800003900144E0FBA3E0FAA3E0F912043CEF51
:103290002401FFE43EFEE43DFDE43CFC12048C907E
:1032A00001507401F0A37401F0A37448F090014739
:1032B0007408F0900147E0609F900150E0FBA3E0AC
:1032C000FAA3E0F9120104FF1256F1900150E0FB5D
:1032D000A3E475F0011201A6A9F0FA120104252950
:1032E000F529900147E014F080C9AF291256F11278
:1032F00058DA227B017A01793C124DECEF60037FB2
:1033000002227B017A01793C12387AC0079002656B
:10331000E0FCA3E0FDA3E0FEA3E0FF90013CE0F8A9
:10332000A3E0F9A3E0FAA3E0FBC312040440047E87
:103330000180027E00D0E04EFFC007900265E0FCF5
:10334000A3E0FDA3E0FEA3E0FF900140E0F8A3E0CE
:10335000F9A3E0FAA3E0FBC312040440047E018059
:10336000027E00D0E04E60037F022212390FA804D3
:10337000A905AA06AB07900265E0FCA3E0FDA3E067
:10338000FEA3E02416FFEE34FCFEED34FFFDEC342A
:10339000FFFCD312040440047F0480027F00227FDC
:1033A0006D1252127F0D1256F1740D2529F5297FE9
:1033B0001E1256F1741E2529F5297F101256F1743C
:1033C000102529F5297F3E1256F1743E2529F5294D
:1033D0007F801256F174802529F5297F641256F1F9
:1033E00074642529F529E4FF1256F17F011256F184
:1033F00005297F401256F174402529F5297F0E12C8
:1034000056F1740E2529F5297F271256F1742725C8
:1034100029F5297F101256F174102529F5299002FB
:10342000B3E025E0FF1256F19002B3E025E0252934
:10343000F5297F201256F174202529F529FF12560F
:10344000F11258DA229001437401F0A37400F0A342
:1034500074A3F0EF90578793FF7E00900148EEF041
:10346000A3EFF0D394497480948040037F012290AD
:10347000014874FFF5F01201A6FED3E5F09400EECA
:103480006480948040361240CD900146EEF0A3EF68
:10349000F0BEFF08BFFF057EFF7FFF22900147E0DF
:1034A0002529F529E0FF900143E0FBA3E475F00135
:1034B0001201A6A9F0FAEF12014A80B31240CD9092
:1034C0000146EEF0A3EFF0BEFF08BFFF057EFF7FD1
:1034D000FF22900146E07004A3E0652960057EFFAD
:1034E0007FFE227E007F0022900146EFF0E49001F3
:1034F00048F0120104FFC4540F900147F0900001FE
:1035000012011DFD7C00EF540FFEE42D90014AF0E6
:10351000EC3E900149F0900147E064067031900163
:1035200049E0FEA3E0FFC394A0EE940F4006BE0F57
:103530001EBFFF1B900146E0FFE4FD1224AD7B019E
:103540007A02790F900146E0FD7C001257512290DB
:103550000147E064077030900149E0FEA3E0FFC33B
:1035600094A0EE940F4006BE0F1DBFFF1A900146B7
:10357000E0FF7D011224AD7B017A02790F900146B4
:10358000E0FD7C0012575122900178EEF0A3EFF09D
:10359000A3EBF0A3EAF0A3E9F0201E29900178E064
:1035A000FEA3E0FFA3E0FBA3E0FAA3E0F91201040D
:1035B000FDC3648094804006EDF4FDFB80027B0037
:1035C000E4FD124A1590017BE475F0011201909020
:1035D000017D7401F090017DE0FDC39421503F9086
:1035E000017AE0FBA3E0FAA3E0F9120104C36480CE
:1035F00094804022900178E0FEA3E0FFA3E0A3E4E2
:1036000075F0011201A6A9F0FA120104FB124A1585
:10361000EF60037F012290017DE004F080B77F001E
:1036200022900151EEF0A3EFF0A3ECF0A3EDF0A394
:10363000EBF0A37403F0900153E09001F2F09001DD
:1036400054E09001F3F0900155E09001F4F0900106
:1036500051E0FEA3E0FF90015D7401F0A37401F05E
:10366000A374F2F07B037D281230D1900151E0FE6B
:10367000A3E0FF90015F7401F0A37401F0A37457FD
:10368000F0A37401F0A37401F0A37458F07B017AE5
:103690000179F27D0F121D20EF700E900157E0B4FA
:1036A00028047F0080027F0222900156E014F0E09F
:1036B000D3940050817F01229002ABEBF0A3EAF09B
:1036C000A3E9F0A3EDF07E007F0B7D001205A3902F
:1036D00002AEE024FE602904707390028174FFF052
:1036E000A37459F0A3740BF0E4A3F0A3F0A3740B3C
:1036F000F09002ABE0FBA3E0FAA3E0F912449A22B7
:1037000090028174FFF0A37459F0A3740FF0E4A346
:10371000F0A3F0A3740BF09002ABE0FBA3E0FAA3DC
:10372000E0F912449A229002AEE075F00BA4243620
:10373000FFE5F03460FEE4FCFD9002ABE0FBA3E0AB
:10374000FAA3E0F990019E740BF0121FE22290029E
:10375000AFEBF0A3EAF0A3E9F0A3EDF07E007F0B5E
:103760007D001205A39002B2E024FE60290470736C
:1037700090028174FFF0A37459F0A37413F0E4A3D2
:10378000F0A3F0A3741FF09002AFE0FBA3E0FAA354
:10379000E0F912449A2290028174FFF0A37459F068
:1037A000A3741BF0E4A3F0A3F0A3741FF09002AF86
:1037B000E0FBA3E0FAA3E0F912449A229002B2E0FF
:1037C00075F01FA42438FFE5F03460FEE4FCFD90A2
:1037D00002AFE0FBA3E0FAA3E0F990019E741FF0B2
:1037E000121FE222EFC39420503774D22FF582E4E7
:1037F0003401F583E07003023879E014F0707A74D4
:10380000B12FF582E43401F583E0606DE4F0EFFD63
:103810007C00E4900158F0A3F0FBFA7FF2124A6BAF
:1038200022E4900146F0900146E0FFC39420504905
:1038300074D22FF582E43401F583E06034E014F0B3
:10384000702F74B12FF582E43401F583E06022908B
:103850000146E0FF24B1F582E43401F583E4F0EFA2
:10386000FD7C00E4900158F0A3F0FBFA7FF2124ACD
:103870006B900146E004F080AD22900196EBF0A33E
:10388000EAF0A3E9F0E4FFA3F0A3F0900196E0FBD7
:10389000A3E0FAA3E0F975F002EFA4F58285F083C6
:1038A0001201E7FDACF090019AE02DF0900199E053
:1038B0003CF00FEFB406D4900199E07002A3E070E1
:1038C00047900196E0FBA3E0FAA3E0F912043C90D4
:1038D0000265E0F8A3E0F9A3E0FAA3E0FBD3120449
:1038E000044025900196E0FBA3E0FAA3E0F99000E4
:1038F0000412045C900265E0F8A3E0F9A3E0FAA3E7
:10390000E0FBD312040450047F0180027F00227B7D
:10391000017A01794F124DEC90014FE0FCA3E0FDDC
:10392000A3E0FEA3E0FFA3E0F8A3E0F9A3E0FAA37D
:10393000E0FBD3120404404190014FE0FCA3E0FD02
:10394000A3E0FEA3E0FF900265E0F8A3E0F9A3E0A6
:10395000FAA3E02FFFEA3EFEE93DFDE83CFC9001C2
:1039600053E0F8A3E0F9A3E0FAA3E0C3EF9BFFEE76
:103970009AFEED99FDEC98FC22900153E0F8A3E04B
:10398000F9A3E0FAA3E0FB90014FE0FCA3E0FDA364
:10399000E0FEA3E0C39BFFEE9AFEED99FDEC98FCE0
:1039A00022900132EDF0EFC39420503CE0FE74B160
:1039B0002FF582E43401F583EEF0EE14600F04700D
:1039C0001974D22FF582E43401F583E4F074D22F18
:1039D000F582E43401F583740AF074D22FF582E4A1
:1039E0003401F5837405F0227E007F20900132E0DF
:1039F000FD7B017A0179B11205A3900132E01460D8
:103A00001204701E7E007F207D007B017A0179D236
:103A10001205A37E007F207D0A7B017A0179D212F4
:103A200005A37E007F207D057B017A0179D21205F6
:103A3000A322EFC39420503174D22FF582E43401D5
:103A4000F583740AF074B12FF582E43401F583E054
:103A5000706D04F0EF4480FD7C00E4900158F0A309
:103A6000F0FBFA7FF2124A6B22E4900146F09001DB
:103A700046E0FFC39420504774D22FF582E434010E
:103A8000F583740AF074B12FF582E43401F583E014
:103A90007025900146E0FF24B1F582E43401F583FE
:103AA0007401F0EF4480FD7C00E4900158F0A3F035
:103AB000FBFA7FF2124A6B900146E004F080AF22DD
:103AC000EF24FE602614603C1460521460682404E5
:103AD000707BED6003B40106ED24FFB3921FEB6031
:103AE0000464017068EB24FF921522ED6003B401B9
:103AF00006ED24FFB39220EB60046401704FEB24C9
:103B0000FF921622ED6003B40106ED24FFB392216B
:103B1000EB600464017036EB24FF921722ED600322
:103B2000B40106ED24FFB39223EB60046401701D21
:103B3000EB24FF921822ED6003B40106ED24FFB3DD
:103B40009224EB6003B40105EB24FF9219224F4B42
:103B5000004154440000434F4E4E454354004A50E8
:103B600031004A5032004A5033004A50340050412C
:103B700053533D3F0041545A002043505220766534
:103B8000722E33302E31362020284329526F67653C
:103B90007220532E432E2020476F736369737A651A
:103BA000776F2D4D616C626F726B20202074656C95
:103BB0002E2F6661782E20302D3535203237323069
:103BC000313233202020687474703A2F2F77777742
:103BD0002E726F6765722E706C00787FE4F6D8FDE8
:103BE000758129023C210210FFE493A3F8E493A31A
:103BF0004003F68001F208DFF48029E493A3F8542F
:103C000007240CC8C333C4540F4420C8834004F4B1
:103C100056800146F6DFE4800B01020408102040C4
:103C200080905AE4E47E019360BCA3FF543F30E5EA
:103C300009541FFEE493A360010ECF54C025E06039
:103C4000A840B8E493A3FAE493A3F8E493A3C8C507
:103C500082C8CAC583CAF0A3C8C582C8CAC583CAF8
:103C6000DFE9DEE780BE900146EFF0120104FFC4F9
:103C7000540FFE900147F0BE0E1A90000112011D74
:103C8000FD7C00EF540FFEE42D900264F0EC3E90BA
:103C90000263F022900147E0640C704B120104545F
:103CA0000F640E704290000112011DFC543F641C11
:103CB0007035900263E0FEA3E0FFC394A0EE940F82
:103CC0005025900146E0FDEC54C0FCBC8003D3803D
:103CD00001C3922A1215037B017A02790F900146E3
:103CE000E0FD7C0012575174FF900263F0A3F022B4
:103CF000900150EBF0A3EAF0A3E9F07B017A01799F
:103D000053124DEC900153E0FCA3E0FDA3E0FEA3B1
:103D1000E0FF900269E0F8A3E0F9A3E0FAA3E0FB7A
:103D2000C3120404700F900150E0FBA3E0FAA3E07B
:103D3000F9125AB522900269E0FCA3E0FDA3E0FE6F
:103D4000A3E0FF900150E0FBA3E0FAA3E0F91250DA
:103D5000679002691204EA900265E0F8A3E0F9A313
:103D6000E0FAA3E0FBD3120404500A9002691205A2
:103D70002B000000007F0022900150EBF0A3EAF03E
:103D8000A3E9F07B017A017953124DEC900153E0E5
:103D9000FCA3E0FDA3E0FEA3E0FF90026DE0F8A32A
:103DA000E0F9A3E0FAA3E0FBC3120404700F900152
:103DB00050E0FBA3E0FAA3E0F9125AB52290026D9D
:103DC000E0FCA3E0FDA3E0FEA3E0FF900150E0FBD8
:103DD000A3E0FAA3E0F912506790026D1204EA9092
:103DE0000265E0F8A3E0F9A3E0FAA3E0FBD3120434
:103DF00004500A90026D12052B000000007F002283
:103E0000900183EEF0A3EFF0A3EDF0A3EBF0E4FF5D
:103E10001259ECE49001D1F07F091256F19001D1D2
:103E2000E02409F0900183E0FF1256F1900183E055
:103E3000FF9001D1E02FF0900184E0FF1256F19045
:103E40000184E0FF9001D1E02FF0900185E0FF12A6
:103E500056F1900185E0FF9001D1E02FF0900186AE
:103E6000E0FF1256F1900186E0FF9001D1E02FF0C3
:103E7000E0FF1256F17F061256F17E007F0022907D
:103E80000143EFF0A3ECF0A3EDF0A3EBF0A3EAF015
:103E9000A3E9F0EF047005E4900143F0900143E0E2
:103EA00004F0E0FED39401501B900149E0FDC3E40F
:103EB0009DFD74649400FCD3900145E09D90014405
:103EC000E09C40037FFF22EE7F00C43333335480F5
:103ED000FEE4AA06900144E0FEA3E0FFE42FFFEA1F
:103EE0003EFEE433FDE433FCA3E0FBA3E0FAA3E0F1
:103EF000F9A3E09001A1F01216E97F002290015091
:103F0000EFF0A3EDF0EFC3942040037F0122900176
:103F100051E060067C007D0180047C007D00900102
:103F200050E0FF900158E4F0A3EFF0E4FBFA7FF6D5
:103F3000124A6BE4900152F0900152E0FFC39420CA
:103F4000502F74002FF582E43400F583E0FE9001D9
:103F500050E0FDEEB50512A3E06003D38001C392EB
:103F60002A900153EFF0125124900152E004F080A6
:103F7000C77F0022900143EFF0A3ECF0A3EDF0A384
:103F8000EBF0A3EAF0A3E9F0EF047005E49001433D
:103F9000F0900143E004F0E0FED39401500E900154
:103FA00045E09400900144E0946440037FFF22EEDA
:103FB0007F00C43333335480FEE4AA06900144E00A
:103FC000FEA3E0FFE42FFFEA3EFEE433FDE433FC12
:103FD000900149E090019EF0900146E0FBA3E0FAD9
:103FE000A3E0F9121FE27F0022900143EFF0125785
:103FF000AC7F6A125212900143E0FF14F0EF60525E
:104000007B017A017945123CF090014D7401F0A3D7
:104010007401F0A37445F09001447408F0900144D9
:10402000E0FF14F0EF60CF90014DE0FBA3E0FAA3B6
:10403000E0F9120104FF1256F190014DE0FBA3E4F8
:1040400075F0011201A6A9F0FA1201042529F5293B
:1040500080CBAF291256F11258DA22900143EFF0CB
:1040600012281B7F75125212900143E0FF14F0EFEB
:1040700060527B017A017945123D7890014D7401BF
:10408000F0A37401F0A37445F09001447408F0901B
:104090000144E0FF14F0EF60CF90014DE0FBA3E09E
:1040A000FAA3E0F9120104FF1256F190014DE0FB72
:1040B000A3E475F0011201A6A9F0FA120104252962
:1040C000F52980CBAF291256F11258DA229002B7A7
:1040D000E014601914603124027048125647EF60F2
:1040E00007C298AF997E00227EFF7FFF229002B622
:1040F0007419F020980B9002B6E070F77EFF7FFFF6
:1041000022C298AF997E00229002B6747DF020986A
:104110000B9002B6E070F77EFF7FFF22C298AF9946
:104120007E00229002B67420F020980B9002B6E038
:1041300070F77EFF7FFF22C298AF997E0022900128
:10414000A312051F9001A3E0FCA3E0FDA3E0FEA3E2
:10415000E0FF7808120415EFFBEEFAE4F9F890029C
:10416000B4E0FEA3E0FFE4FCFDC31203EE603E12E8
:104170005872C2849001A3E0FCA3E0FDA3E0FEA37B
:10418000E0FF9001AD12051F7F53121E88D284906C
:1041900001A3E0FCA3E0FDA3E0FEA3E0FF7808128A
:1041A0000415EFEEE49002B4EEF0A3EFF0229001DC
:1041B00043EFF0C364809480500E7F061258057F51
:1041C000D07E0712596980F2900143E0700204F03A
:1041D000900143E0FF9002B8F03395E0FEFDFCF85B
:1041E000F9FAAB07E47F34FEFDFC124FA0AD07AC3B
:1041F00006C3E49DFDE49CFCE4F5C8C2ADC2ACEC92
:10420000FFF5CBAE05EEF5CA8FCDF5CC759853C250
:1042100098D29975C8349002B77402F022204350A6
:1042200052207665722E33302E31362020284329D5
:10423000526F67657220532E432E2020476F7363A1
:1042400069737A65776F2D4D616C626F726B202098
:104250002074656C2E2F6661782E20302D35352028
:1042600032373230313233202020687474703A2F64
:104270002F7777772E726F6765722E706C006400EF
:10428000660076000000A2C200000034900198EBA6
:10429000F0A3EAF0A3E9F0AC05AD07EC605A125ABE
:1042A0008AED54F04402FF12583E90019BE0FF1249
:1042B000583E125A8AED54F04403FF12583E1CEC4B
:1042C000601C125858900198E0FBA3E475F00112AD
:1042D00001A6A9F0FAEF12014A125B0E80E0125813
:1042E00058900198E0FBA3E475F0011201A6A9F033
:1042F000FAEF12014A125AA822900196EBF0A3EAB3
:10430000F0A3E9F0900196E0FBA3E0FAA3E0F91234
:10431000043C900265E0F8A3E0F9A3E0FAA3E0FB17
:10432000D31204045012900196E0FBA3E0FAA3E03C
:10433000F912055C00000000900196E0FBA3E0FA92
:10434000A3E0F912043C9000041204A6900008E4D3
:10435000F5F01202A490000412045C9002691205A8
:104360001F22E4900132F0900132E0FFC364809498
:10437000A050577B017A02790FEFFD3395E0FC12D4
:10438000575190020FE0FEA3E0FF90013BEEF0A337
:10439000EFF04E602D90013BE0FEA3E0FF7B017A41
:1043A000017933123196EF7019900133E0FFC45454
:1043B0000F600F90013BE0FEA3E0FFE4FD124E8191
:1043C00080D3900132E004F0809D2290029CEBF0BB
:1043D000A3EAF0A3E9F0A3EDF0A3E0FDC3648094A9
:1043E00080404D90029FE0702A201E2790029CE0A2
:1043F000FBA3E0FAA3E0F91201BCFFAEF0C3ED6449
:104400008094804006EDF4FDFB80027B00E4FD1209
:104410004A152290029CE0FBA3E0FAA3E0F9120106
:10442000BCFFAEF090029FE0FDA3E0FB124A152214
:104430007F0122900287EBF0A3EAF0A3E9F090025B
:104440008AE0FBA3E0FAA3E0F9120104FE900287E0
:10445000E0FBA3E0FAA3E0F9120104FD6E702AED7F
:10446000600E90028D74FFF5F012019045F070031C
:104470007F0022900288E475F00112019090028B77
:10448000E475F00112019080B5D3EE6480F8ED641C
:10449000809840037F01227FFF2290027EEBF0A3F1
:1044A000EAF0A3E9F0900285E07002A3E0604B908F
:1044B0000281E0FBA3E475F0011201A6A9F0FA1253
:1044C0000104FF90027EE0FBA3E475F0011201A657
:1044D000A9F0FAEF12014A900284E06F700C90028A
:1044E0007EE0FBA3E0FAA3E0F922900286E024FF3D
:1044F000F0900285E034FFF080AB7B007A00790019
:1045000022125A6A900132EFF0BFFF0E7F0212585A
:10451000057FE87E0312596980E7900132E0543844
:1045200024E8601024F06014242070189002B37402
:1045300002F0802A9002B37408F080229002B374D3
:1045400020F0801A7F021258057FF47E011259690B
:104550007F021258057F887E1312596980E6900207
:10456000B3E0FF227B017A017943124DEC900143C5
:10457000E0FCA3E0FDA3E0FEA3E0FFA3E0F8A3E0DE
:10458000F9A3E0FAA3E0FBC31204046037900147EB
:104590001204EA900265E0F8A3E0F9A3E0FAA3E0D0
:1045A000FBD3120404500A90014712052B000000AF
:1045B00000E490014BF0A3F07B017A0179431251A2
:1045C000DA7F00227F0122900199EBF0A3EAF0A3A9
:1045D000E9F0E4FFA3F0A3F0900199E0FBA3E0FA77
:1045E000A3E0F975F002EFA4F58285F0831201E7EC
:1045F000FDACF090019DE02DF090019CE03CF00FAF
:10460000EFB405D490019CE0FEA3E0FFC3E49FFF5C
:10461000E49EFE900199E0FBA3E0FAA3E0F990008C
:104620000AEE8FF01202A422AD07AC06900143748B
:10463000FFF0A3742CF0A37448F0E4A3F0900143BE
:10464000E0FBA3E0FAA3E0F91201BCFFC3ED9FEC8D
:1046500095F050089000021201E7FF22900144E417
:1046600075F004120190900146E004F0E0B442CDF0
:10467000900143E0FBA374FF75F0FC120190A9F0D8
:10468000FA9000041201E7FF22D286A2A4922AD255
:10469000A47F017E00125969C28E53890F4389108D
:1046A000E4F58BF58DC28FC2AFC2A4D28E208603F3
:1046B000308FFAC28ED2AFA22A92A4AF8DEFFEAD98
:1046C0008B7C00E42DFFEC3EAD07FC208F09D3ED81
:1046D00094FFEC947F40057EFF7FFF22AE04AF0580
:1046E000ED25E0FFEC33FE229002A1EBF0A3EAF00F
:1046F000A3E9F0A3EDF09002B77403F01240CDC32C
:10470000EE648094804028EF9420EE648094804092
:10471000269002A1E0FBA3E475F0011201A6A9F026
:10472000FAEF12014A9002A4E014F0600A80CD90E2
:1047300002A5E014F070C59002A1E0FBA3E0FAA38B
:10474000E0F9E412014A22201F047F0180027F0069
:10475000301504EF4402FF202004EF4404FF30161C
:1047600004EF4408FF202104EF4410FF301704EF4A
:104770004420FF202304EF4440FF301804EF44801E
:10478000FFEF12014A2024047E0180027E00AF0662
:10479000301904EF4402FF20A704EF44C0FF90004B
:1047A00001EF12015C229002BFEBF0A3EAF0A3E953
:1047B000F0E4FF1259EC9002BFE0FBA3E0FAA3E0A3
:1047C000F91250267F011259EC7B017A0279379059
:1047D00002A57402F07D101246E87BFF7A3B794E09
:1047E0001259C390028DEEF0A3EFF090028A74FF8D
:1047F000F0A3743BF0A3744EF07B017A0279371278
:104800004433227FFF124ECBEF60037F02227B01F5
:104810007A01793212224E900137E0D3943B50282E
:10482000900136E0943B5020900135E094175018E9
:10483000900134E0941F5010900133E0940C500824
:10484000900132E0946340037F04221232F3EF249C
:10485000FC6007240270067F03227F05227F00226E
:10486000300A13C20AE4900158F0A3F0FBFA7D0667
:10487000FC7FF1124A6B302613C226E4900158F0F7
:10488000A3F0FBFA7D05FC7FF1124A6B300E13C2D8
:104890000EE4900158F0A3F0FBFA7D0AFC7FF112C0
:1048A0004A6B300B13C20BE4900158F0A3F0FBFAF3
:1048B0007D09FC7FF1124A6B227F301256CF7F01B7
:1048C0001259EC9002B77401F012064DEE703FEFF2
:1048D000249F703A9001327403F0A374E8F09001C1
:1048E00032E0FEA3E0FFF47002EEF4601EEF6462BB
:1048F0004E60189002B77402F012064D900132EE2D
:10490000F0A3EFF07F011259EC80D37F01227F00EA
:1049100022900143EFF0C3940140037FFF229001F6
:1049200043E0FF124ECBEF60037FFE22E490014490
:10493000F0900144E0FFD39464502AEFFD7C007EA8
:1049400000C007900143E075F080A4FF2480FFE4DD
:1049500035F0CF2DFDEC3FFCD00712550E900144F1
:10496000E004F080CC7F00229002A6EFF0A3EDF0EF
:10497000A3EBF0A3EAF0A3E9F0E4FF1259EC9002F4
:10498000A6E0FF6004F599800375993D7F0A7E00DB
:104990001259699002A7E0FF14F0EF601CA3E0FB3E
:1049A000A3E475F0011201A6A9F0FA120104F59929
:1049B0007F0A7E0012596980DA7F011259EC229039
:1049C00001A312051F125872C2849001A3E0FCA338
:1049D000E0FDA3E0FEA3E0FF9001AD12051F7F8480
:1049E000121E889001A774FFF5F01201A645F06031
:1049F000199001A9E0FBA3E475F0011201A6A9F04A
:104A0000FA120104FF125A4880D9D28474FF90022E
:104A1000B4F0A3F02290017EEEF0A3EFF0A3EDF04E
:104A2000A3EBF0A37403F090017EE0FEA3E0FFA3EC
:104A3000E0FD25E0FDA3E054014DFB7D44123E0066
:104A400090017EE0FEA3E0FF900187E4F0A3F0A3D5
:104A5000F0FB7D441225D6EF7002FF22900182E028
:104A600014F0E0D3940050BF7F0122900153EFF087
:104A7000A3ECF0A3EDF0A3EAF0A3EBF07B017A0145
:104A8000795A12224E900153E0900162F090015544
:104A9000E0900163F0900157E0900164F0900159BB
:104AA000E0900165F090017C7401F0A37401F0A323
:104AB0007462F07B017A01795A7FFF12188F22907D
:104AC0000154EEF0A3EFF0ED54074428900157F0A5
:104AD0009001567403F0900154E0FEA3E0FF9001B2
:104AE00057E0FB7D4B123E00900154E0FEA3E0FF37
:104AF000900187E4F0A3F0A3F0FB7D4B1225D6EFE5
:104B00007002FF22900156E014F0E0D3940050C6EA
:104B10007F0122900178EEF0A3EFF0ED5407448876
:104B200090017BF090017A7403F0900178E0FEA38D
:104B3000E0FF90017BE0FB7D4B123E00900178E0AE
:104B4000FEA3E0FF900187E4F0A3F0A3F0FB7D4B10
:104B50001225D6EF7002FF2290017AE014F0E0D324
:104B6000940050C67F0122900178EEF0A3EFF0EDA3
:104B70005407448090017BF090017A7403F0900117
:104B800078E0FEA3E0FF90017BE0FB7D4B123E004E
:104B9000900178E0FEA3E0FF900187E4F0A3F0A38A
:104BA000F0FB7D4B1225D6EF7002FF2290017AE0D8
:104BB00014F0E0D3940050C67F01229001A01205AA
:104BC0001F125872C2849001A0E0FCA3E0FDA3E094
:104BD000FEA3E0FF9001AD12051F7F54121E88E472
:104BE000FF125A489001A474FFF5F01201A645F097
:104BF00060191259979001A6E0FBA3E475F0011229
:104C000001A6A9F0FAEF12014A80D9D284229001BC
:104C1000457401F0A37402F0A37401F0E4FF900165
:104C200043F0A3F0900145E0FBA3E475F00212010C
:104C3000A6A9F0FA1201BCFDACF0900144E02DF001
:104C4000900143E03CF00FEFB406D9900143E0FE41
:104C5000A3E0FFC3E49FFFE49E90020DF0A3EFF0FA
:104C6000227B017A017943124DEC900269E0FCA3AA
:104C7000E0FDA3E0FEA3E0FF900147E0F8A3E0F928
:104C8000A3E0FAA3E0FBC31204046007E490014B25
:104C9000F0A3F0900269E0FCA3E0FDA3E0FEA3E036
:104CA000FF90014712051F7B017A0179431251DA07
:104CB0007F0022900148EEF0A3EFF0A3EDF0E4FCBA
:104CC000FD780812042912413E125872C2849001E4
:104CD00048E0FEA3E0FFE4FCFD78081204299001FF
:104CE000AD12051F7F54121E88E4FF125A48E4FDDE
:104CF000125997EF2DFD90014AE014F070F2D28422
:104D0000AF0522900153EBF0A3EAF0A3E9F0900184
:104D100053E0FBA3E0FAA3E0F912043C900265E043
:104D2000F8A3E0F9A3E0FAA3E0FBD3120404401FC8
:104D3000900153E0FBA3E0FAA3E0F912043C9001D8
:104D400056E0FBA3E0FAA3E0F91250677F00227F50
:104D500005229001347401F0A37402F0A37401F0F1
:104D6000E4FF900132F0A3F0900134E0FBA3E4757E
:104D7000F0021201A6A9F0FA1201BCFDACF09001FC
:104D800033E02DF0900132E03CF00FEFB407D99002
:104D90000132E07002A3E060047F0180027F002204
:104DA000301D48C21D125483900132EFF0D2819021
:104DB00002C3E06F6015900132E0FD7C00E49001D9
:104DC00058F0A3F0FBFA7FF1124A6B900132E0FF3A
:104DD000B40803D38001C3922220220A9002C3E0C8
:104DE000B408037518FA9002C3EFF022900193EB18
:104DF000F0A3EAF0A3E9F090019B7420F07D0C7F12
:104E0000A012428C900193E0FBA3E0FAA3E0F91218
:104E1000387AEF601F900193E0FBA3E0FAA3E0F97A
:104E20001242F9900193E0FBA3E0FAA3E0F91251DA
:104E3000DA7F01227F002290019312051F900197D3
:104E4000EBF0A3EAF0A3E9F0E47F08FEFDFC90019B
:104E500093E0F8A3E0F9A3E0FAA3E0FB1202D1E4A7
:104E60002FFFE43EFEED3401FDE43CFC900197E0B1
:104E7000FBA3E0FAA3E0F99001A17408F01216E98F
:104E800022900146EEF0A3EFF0A3EDF0A37403F03F
:104E9000900146E0FEA3E0FFA3E0FB7D42123E004E
:104EA000900146E0FEA3E0FF900187E4F0A3F0A3A9
:104EB000F0FB7D421225D6EF7002FF22900149E0FF
:104EC00014F0E0D3940050C87F0122900145EFF028
:104ED000047005E4900145F0900145E004F0E4A37E
:104EE000F0A3F0900146E0FDC39464502190014589
:104EF000E075F080A47C002DFFEC35F0FE125B1E07
:104F0000900147E02FF0900146E004F080D5900139
:104F100047E0FF22900143EDF0A3EBF0A3EAF0A3FA
:104F2000E9F0125212900143E0FF14F0EF6023A366
:104F3000E0FBA3E475F0011201A6A9F0FA12010446
:104F4000FF900147F01256F1900147E02529F5291D
:104F500080D3AF291256F11258DA229001A312051C
:104F60001F125872C2849001A3E0FCA3E0FDA3E0ED
:104F7000FEA3E0FF9001AD12051F7F83121E88D2B1
:104F8000849001A3E0FCA3E0FDA3E0FEA3E0FF7892
:104F900008120415EFEEE49002B4EEF0A3EFF02255
:104FA000C2D5E830E70FB2D5E4C39BFBE49AFAE43C
:104FB00099F9E498F8EC30E717B2D5124FD61203FE
:104FC0005CE4C39BFBE49AFAE499F9E498F8800363
:104FD00012035C30D50DE4C39FFFE49EFEE49DFD0B
:104FE000E49CFC22125AD9D284C2B7A2B5B392B5BE
:104FF0007F057E00125969A2B5B392B57F057E0088
:10500000125969A2B5B392B57F057E00125969A203
:10501000B5B392B57F057E00125969D2B7A2B5B378
:1050200092B5125AD9229002BCEBF0A3EAF0A3E9A0
:10503000F09002BCE0FBA3E0FAA3E0F912010460E7
:10504000189002BCE0A3E475F0011201A6A9F0FAE1
:10505000120104FF1256F180D87F0D1256F17F0A1B
:105060001256F11258DA2290019312051FC003C0A4
:1050700002C001E47F08FEFDFC900193E0F8A3E08C
:10508000F9A3E0FAA3E0FB1202D1E42FFFE43EFE15
:10509000ED3401FDE43CFC90019E7408F0D001D099
:1050A00002D003121FE222E490028FF0A3F0A3F0DB
:1050B000A3F0A3F0A304F0A3F090019CF0A374026A
:1050C000F0A3748FF0E4FB7D077FA012538A900158
:1050D0009C7401F0A37402F0A3748FF07B3A7D01FD
:1050E0007FA012538A227B017A01797812224E9096
:1050F000017EE0FB7A007C007D18FF7E0012017EBD
:10510000AA06AB0790017BE02BFBE43AFA7D3CAFAB
:1051100003FE12017EAA06AB07A3E02BFBE43AFADA
:10512000FEAF03227B017A02790F900153E0FD7CF0
:105130000012575190020FE0FEA3E0FFF47002EE60
:10514000F4601EEF4E601AA22AE433FD124ABF90AB
:10515000020FE0FEA3E0FFA22AE433FBE4FD124AC3
:105160001522900143EFF0047005E4900143F090A4
:105170000143E004F0E4A3F0900144E0FDD3946423
:10518000501B900143E075F080A47C002DFFEC35AE
:10519000F0FE1253BE900144E004F080DB22900147
:1051A00043EEF0A3EFF0A3EDF0BEFF0CBFFF09E06C
:1051B000B4FF0512578E801F900143E0FCA3E0FD71
:1051C000C394A0EC940F40037FFF22AF05AE049080
:1051D0000145E0FD12558A7F0022900196EBF0A375
:1051E000EAF0A3E9F0900196E0FBA3E0FAA3E0F96E
:1051F0001245C7900196E0F9A3E0FAA3E090019C64
:10520000C9F0A3EAF0A3E9F07B207D0C7FA0125344
:105210008A22900153EFF0E4FF1259EC7F421256BC
:10522000F17F621256F17F131256F1900153E0FFA5
:105230001256F1E4F52974A42529F5292413F5293A
:10524000900153E02529F529229002B9EBF0A3EA59
:10525000F0A3E9F09002B9E0FBA3E0FAA3E0F912B1
:10526000010460189002B9E0A3E475F0011201A6F0
:10527000A9F0FA120104FF1256F180D81258DA226E
:10528000B2B590000075F000E49325F0F5F0A3E5C9
:105290008270F5E583B2B5B460EE85F01DE51D6062
:1052A00014C2A57FB87E0B1258C0D2A57FB87E0B62
:1052B0001258C080EC2290014FEEF0A3EFF07B017A
:1052C0007A02790FED7C0012575190020FE0FEA395
:1052D000E0FFF47002EEF46011EF4E600D90014FAC
:1052E000E0FCA3E0FDE4FB1236212290014FEEF03A
:1052F000A3EFF07B017A02790FED7C0012575190F9
:10530000020FE0FEA3E0FFF47002EEF46011EF4E36
:10531000600D90014FE0FCA3E0FD7B0112362122DD
:1053200090014FEEF0A3EFF07B017A02790FED7C54
:105330000012575190020FE0FEA3E0FFF47002EE5E
:10534000F46011EF4E600D90014FE0FCA3E0FD7B97
:10535000021236212290014FEEF0A3EFF07B017A8A
:1053600002790FED7C0012575190020FE0FEA3E08E
:10537000FFF47002EEF46011EF4E600D90014FE00B
:10538000FCA3E0FD7B0312362122ED6030125A8A25
:10539000EF54F04402FF12583EAF0312583E900102
:1053A0009CE0FBA3E475F0011201A6A9F0FA12013A
:1053B00004FF12583EDDE7125AA81258F32290015A
:1053C00047EEF0A3EFF0125872C284900147E0FE5E
:1053D000A3E0FFE4FCFD78081204299001AD12055A
:1053E0001F7F81121E88D28474FF9002B4F0A3F054
:1053F000229001ACEFF09001ACE0601AC2A57FC82A
:105400007E00125969D2A57FC87E001259699001A9
:10541000ACE014F080E07FD07E07125969A2B5B3EA
:1054200092B522ED75F021A4FF90017CE07C002F65
:10543000FFEC35F0FEEF7802C333CE33CED8F9243B
:1054400041FFEE344FFEE4FCFD90019E7404F01227
:105450001FE222900143EEF0A3EFF0A3EDF0E4FB96
:105460007D45123E00900143E0FEA3E0FF900187DE
:105470007401F0A37401F0A37446F07B017D451222
:1054800025D622124689AD07AC06D281D3ED9467AA
:10549000EC940D40037F0D22D3ED941FEC940C404F
:1054A000037F0722D3ED9420EC940340037F08226E
:1054B0007F0D22900143EFF02DFFE43CFED3EF94EB
:1054C000A0EE940F40037FFF22E42DFFEC3466FE34
:1054D000E4FCFD900143E090019EF0121FE27F008A
:1054E000227B017A027948125A1290024874C3F062
:1054F000E4A3F0A37420F0A37403F0741EF0A3746B
:1055000001F0125AC19228D291D280C2A5229001F4
:1055100045EEF0A3EFF0AE04AF05E4FCFD78081211
:10552000042912413E900145E0FEA3E0FFE4FCFDAA
:105530007808120429124F5B22ED75F004A4FDAC2B
:10554000F090017CE075F080A4FF2DFFE5F03CCFEA
:1055500024A0CF3460FEE4FCFD90019E7404F012A0
:105560001FE2229001A312051F125872C2849001FB
:10557000A3E0FCA3E0FDA3E0FEA3E0FF9001AD12D9
:10558000051F7F58121E88D2842290014FEDF0C370
:10559000EF94A0EE940F5018E42FFFEE3466FEE473
:1055A000FCFD7B017A01794F9001A104F01216E90C
:1055B00022900201E0FF13B39210EFA2E19225A224
:1055C000E2921EA2E39214A2E49212A2E59202A237
:1055D000E6921B33920322124501EF24FFFFE434CD
:1055E000FFFEE4FCFDFBFA7901F81202D1E47B082E
:1055F000FAF9F8124FA090026512051F2212064D0B
:10560000900133EEF0A3EFF07F011259EC900133DB
:10561000E0FEA3E0FFF47002EEF46006EF64624E79
:1056200070DB22900132EFF01256697FD07E0712B4
:105630005969D206900132E0FF125805E4FF124189
:10564000AE1255FD80FB22C28E53890F438910751F
:105650008BEB758DCBC28FD28E209808308FFAC21B
:105660008E7F0022C28E7F01227E007F0E7D007B16
:10567000017A0279011205A37E007F027DFF7B0182
:105680007A0279011205A312577022900143EFF0BC
:105690007F2B125212900143E0FF1256F19001430A
:1056A000E02529F529FF1256F11258DA229001431C
:1056B000EFF07F2D125212900143E0FF1256F1904D
:1056C0000143E02529F529FF1256F11258DA2290FC
:1056D0000134EFF07F3F125212900134E0FF125676
:1056E000F1900134E02529F529FF1256F11258DA1C
:1056F00022AD079002B67404F020990B9002B6E038
:1057000070F77EFF7FFF22C299AF058F997E007FE1
:105710000022900143EDF0125212900143E0FF127B
:1057200056F1900143E02529F529FF1256F1125850
:10573000DA22E49002C4F09002C4E0FFC3648094D3
:10574000A0500B120C4A9002C4E004F080E97F00E4
:1057500022AE04ED7802C333CE33CED8F924A1FFB4
:10576000E43EFEE4FCFD90019E7404F0121FE22270
:105770001255B1124C0E90019C7401F0A37402F00A
:10578000A37401F07B2C7D0E7FA012538A2290011E
:10579000467466F0900146E0FFC39476500D7E009B
:1057A0001253BE900146E004F080E9227B017A01A9
:1057B0007950124DEC900154E0FCA3E0FDA3E0FE13
:1057C000A3E0FF90026912051F227B017A01794351
:1057D000124DEC7B017A0179431242F97B017A0187
:1057E00079431251DA7F00220000070001034301D0
:1057F000000101000000000C00040101050000058B
:105800000108000303AD07AF051DEF6014C2A57FBB
:10581000647E00125969D2A57FC87E001259698042
:10582000E622ED25E0FFEC33FEEF2421FFEE34010C
:10583000FEE4FCFD90019E7402F0121FE2227E083D
:10584000EF339296D297EF25E0FFC297DEF2C29631
:1058500000D2970000C29722D2967E08C29712000B
:105860000AD297EF25E0FDA296E4334DFFDEEDC2AC
:105870009722125AD97DC8125A6AEFF46004EF20B9
:10588000E709DDF37F021253F180F9227B017A02EE
:10589000790190019B742CF07D0E7FA012428C1236
:1058A00055B1124D5222EF75F002A424C1FFE5F06C
:1058B000345FFEE4FCFD90019E7402F0121FE222B0
:1058C000AB07AA06EB1BAE0270011A4E600BB2B515
:1058D0007F017E0012596980EB229002B67404F0B9
:1058E00020990B9002B6E070F77EFF7FFF227E00CA
:1058F0007F0022C28E53890F438910758BEB758D03
:10590000CBC28FD28E308FFDC28E224141410042E8
:105910004242003637313536363100363731353987
:10592000313000C28E53890F438910758BCB758D32
:10593000FAC28FD28E308FFDC28E227F011259ECB7
:105940009002B77401F01240CDBEFFFABFFFF77F9F
:1059500001226A50202D20706C204D6F6E61204C0A
:10596000697361203230303100EF1FAC0670011EC8
:10597000D39400EC64809480400512592380EA227D
:10598000C2AF5389F0438901758A3E758C5DC2B9F7
:10599000D2A9D28CD2AF227F08E4FEC297EE25E0D6
:1059A000FE3082010ED29700DFF1AF06227F011296
:1059B00059ECE49002B7F01240CDBEFFFABFFFF7FA
:1059C0007F0122E4FFFE120104600C0FEF70010E54
:1059D00009E970F20A80EF22EF75F00A84FEC454E0
:1059E000F0FEEF75F00A84E5F04EFF22EF700BD267
:1059F00093C2B67F03FE12596922D2B6C293227BAC
:105A0000017A007962125A247B017A007900125AD5
:105A1000362290019E740BF07F957E607D007C00A5
:105A2000121FE22290019E7440F07FC17E5F7D00D4
:105A30007C00121FE22290019E7440F07F017E6084
:105A40007D007C00121FE2227E08EF339283C29712
:105A5000EF25E0FFD297DEF2221201BCFFAEF090FC
:105A6000000212011DFD12545322125AD9C2847F22
:105A700057125A48125997D284227E007F047D0023
:105A80007B017A0279331205A322D296D2971200B3
:105A90000A00C2960000C29722EFC4540F75F00AA4
:105AA000A4FEEF540F2EFF22C29612000AD29712C4
:105AB000000AD296227E007F087D001205A37F0196
:105AC00022900248E0B4C303D38001C3229002496C
:105AD000E030E003D38001C322D2B7D284D283D294
:105AE00082D297224202B4FFFF420263FFFF0012FC
:105AF00000037FC87E0012596922E4F518D2A7D2AC
:105B0000A5C22722C2AF7F011259EC80FE22C296A5
:105B1000D2970000C297223095FD2095FD22E4FD2A
:105B2000124CB3227F0022D28122FFFFFFFFFFFF32
:105B3000FFFFFFFFFFFFFFFFFFFFFFFFFFFFFFFF75
:105B4000FFFFFFFFFFFFFFFFFFFFFFFFFFFFFFFF65
:105B5000FFFFFFFFFFFFFFFFFFFFFFFFFFFFFFFF55
:105B6000FFFFFFFFFFFFFFFFFFFFFFFFFFFFFFFF45
:105FF000FFFFFFFFFFFFFFFFFFFFFFFFFFFFFF159B
:00000001FF
